:020000020000FC
:020000000EC030
:020006003EC0FA
:10001C0024C00FEF01BB0FEF02BB00E004BB00E3F9
:10002C0005BB0FEF07BB0FEF08BB0FE50DBF04E0DF
:10003C000EBF41E00DE005BD06E203BD00E809BFBF
:10004C0000EE07B90BE806B900E905BF789400E8A3
:10005C0008B9FFCF78948895089505B120E030E079
:10006C00043638F40A3018F00A503395FBCF202FA1
:10007C0002C02FEF3FEF189508D04A9529F442E0C3
:10008C005A9511F452E3E6DF189500E008BB4130B5
:10009C0011F0423031F0022F0AD002BB01E008BB54
:1000AC000895032F04D002BB02E008BB0895003072
:1000BC00A1F00130A1F00230A1F00330A1F0043026
:1000CC00A1F00530A1F00630A1F00730A1F0083006
:1000DC00A1F00930A1F00FEB089500EC089509EFA1
:1000EC00089504EA089500EB089509E9089502E9DA
:1000FC00089502E8089508EF089500E8089500E9CE
:02010C00089554
:00000001FF
